:100000000C29FF3FFF3FFF3F031383120610C3304D
:10001000C000FF30C100C00B0E281128C10B0E28F4
:100020000B284B30C000C00B13280000080003133E
:10003000831206100330C000FF30C100FF30C20041
:10004000C00B23282A28C10B26282928C20B2628C2
:10005000232820284B30C000FF30C100C00B3128BE
:100060003428C10B31282E28DD30C000C00B3628C3
:10007000000008000313831206140330C000FF3091
:10008000C100FF30C200C00B46284D28C10B4928D3
:100090004C28C20B4928462843284B30C000FF306B
:1000A000C100C00B54285728C10B54285128DD30FB
:1000B000C000C00B592800000610042008000313DC
:1000C00083120614C330C000FF30C100C00B692882
:1000D0006C28C10B692866284B30C000C00B6E2805
:1000E00000000610042008005F203A2017200800B6
:1000F0005F20172008005F205F205F205F2017200F
:1001000008003A205F203A201720080003138312CA
:1001100006100630C000FF30C100FF30C200C00B27
:1001200092289928C10B95289828C20B95289228C7
:100130008F285B30C000FF30C100C00BA028A3286F
:10014000C10BA0289D280630C000C00BA5280800C0
:100150000313831206143330C000FF30C100FF3098
:10016000C200C00BB428BB28C10BB728BA28C20BE9
:10017000B728B428B128FD30C000FF30C100C00B43
:10018000C228C528C10BC228BF28B530C000C00B8B
:10019000C7280000061008005F203A203A205F20A0
:1001A000172008005F203A205F20172008003A201F
:1001B0005F205F205F205F20172008003A20172073
:1001C00008005F205F205F203A20172008005F2092
:1001D0003A203A2017200800031383128614A8201F
:1001E0008620E1208120D720D220E720742086209D
:1001F000A8208620CC207820D220DE207B208620DC
:1002000086100800031383128501FF3083168500D2
:100210008601831286010800022103138312C101A3
:100220008519C10A00304102031D1829EC20192943
:1002300086100D291A29FF3FFF3FFF3FFF3FFF3F79
:02400E00FD3F74
:00000001FF
